###############################################################################
#                                                                             #
# IAR ELF Linker V6.70.2.6274/W32 for ARM               02/Oct/2015  15:14:12 #
# Copyright 2007-2013 IAR Systems AB.                                         #
#                                                                             #
#    Output file  =  D:\Projects\MicroTechnics\STM32Cube\STM32Cube_SDCardProj #
#                    ect\EWARM\STM32Cube_SDCardProject                        #
#                    Configuration\Exe\STM32Cube_SDCardProject                #
#                    Configuration.out                                        #
#    Map file     =  D:\Projects\MicroTechnics\STM32Cube\STM32Cube_SDCardProj #
#                    ect\EWARM\STM32Cube_SDCardProject                        #
#                    Configuration/List\STM32Cube_SDCardProject               #
#                    Configuration.map                                        #
#    Command line =  "D:\Projects\MicroTechnics\STM32Cube\STM32Cube_SDCardPro #
#                    ject\EWARM\STM32Cube_SDCardProject                       #
#                    Configuration\Obj\bsp_driver_sd.o"                       #
#                    "D:\Projects\MicroTechnics\STM32Cube\STM32Cube_SDCardPro #
#                    ject\EWARM\STM32Cube_SDCardProject                       #
#                    Configuration\Obj\ccsbcs.o"                              #
#                    "D:\Projects\MicroTechnics\STM32Cube\STM32Cube_SDCardPro #
#                    ject\EWARM\STM32Cube_SDCardProject                       #
#                    Configuration\Obj\diskio.o"                              #
#                    "D:\Projects\MicroTechnics\STM32Cube\STM32Cube_SDCardPro #
#                    ject\EWARM\STM32Cube_SDCardProject                       #
#                    Configuration\Obj\ff.o" "D:\Projects\MicroTechnics\STM32 #
#                    Cube\STM32Cube_SDCardProject\EWARM\STM32Cube_SDCardProje #
#                    ct Configuration\Obj\ff_gen_drv.o"                       #
#                    "D:\Projects\MicroTechnics\STM32Cube\STM32Cube_SDCardPro #
#                    ject\EWARM\STM32Cube_SDCardProject                       #
#                    Configuration\Obj\main.o" "D:\Projects\MicroTechnics\STM #
#                    32Cube\STM32Cube_SDCardProject\EWARM\STM32Cube_SDCardPro #
#                    ject Configuration\Obj\sd_diskio.o"                      #
#                    "D:\Projects\MicroTechnics\STM32Cube\STM32Cube_SDCardPro #
#                    ject\EWARM\STM32Cube_SDCardProject                       #
#                    Configuration\Obj\startup_stm32f103xe.o"                 #
#                    "D:\Projects\MicroTechnics\STM32Cube\STM32Cube_SDCardPro #
#                    ject\EWARM\STM32Cube_SDCardProject                       #
#                    Configuration\Obj\stm32f1xx_hal.o"                       #
#                    "D:\Projects\MicroTechnics\STM32Cube\STM32Cube_SDCardPro #
#                    ject\EWARM\STM32Cube_SDCardProject                       #
#                    Configuration\Obj\stm32f1xx_hal_cortex.o"                #
#                    "D:\Projects\MicroTechnics\STM32Cube\STM32Cube_SDCardPro #
#                    ject\EWARM\STM32Cube_SDCardProject                       #
#                    Configuration\Obj\stm32f1xx_hal_dma.o"                   #
#                    "D:\Projects\MicroTechnics\STM32Cube\STM32Cube_SDCardPro #
#                    ject\EWARM\STM32Cube_SDCardProject                       #
#                    Configuration\Obj\stm32f1xx_hal_flash.o"                 #
#                    "D:\Projects\MicroTechnics\STM32Cube\STM32Cube_SDCardPro #
#                    ject\EWARM\STM32Cube_SDCardProject                       #
#                    Configuration\Obj\stm32f1xx_hal_flash_ex.o"              #
#                    "D:\Projects\MicroTechnics\STM32Cube\STM32Cube_SDCardPro #
#                    ject\EWARM\STM32Cube_SDCardProject                       #
#                    Configuration\Obj\stm32f1xx_hal_gpio.o"                  #
#                    "D:\Projects\MicroTechnics\STM32Cube\STM32Cube_SDCardPro #
#                    ject\EWARM\STM32Cube_SDCardProject                       #
#                    Configuration\Obj\stm32f1xx_hal_gpio_ex.o"               #
#                    "D:\Projects\MicroTechnics\STM32Cube\STM32Cube_SDCardPro #
#                    ject\EWARM\STM32Cube_SDCardProject                       #
#                    Configuration\Obj\stm32f1xx_hal_msp.o"                   #
#                    "D:\Projects\MicroTechnics\STM32Cube\STM32Cube_SDCardPro #
#                    ject\EWARM\STM32Cube_SDCardProject                       #
#                    Configuration\Obj\stm32f1xx_hal_pwr.o"                   #
#                    "D:\Projects\MicroTechnics\STM32Cube\STM32Cube_SDCardPro #
#                    ject\EWARM\STM32Cube_SDCardProject                       #
#                    Configuration\Obj\stm32f1xx_hal_rcc.o"                   #
#                    "D:\Projects\MicroTechnics\STM32Cube\STM32Cube_SDCardPro #
#                    ject\EWARM\STM32Cube_SDCardProject                       #
#                    Configuration\Obj\stm32f1xx_hal_rcc_ex.o"                #
#                    "D:\Projects\MicroTechnics\STM32Cube\STM32Cube_SDCardPro #
#                    ject\EWARM\STM32Cube_SDCardProject                       #
#                    Configuration\Obj\stm32f1xx_hal_sd.o"                    #
#                    "D:\Projects\MicroTechnics\STM32Cube\STM32Cube_SDCardPro #
#                    ject\EWARM\STM32Cube_SDCardProject                       #
#                    Configuration\Obj\stm32f1xx_it.o"                        #
#                    "D:\Projects\MicroTechnics\STM32Cube\STM32Cube_SDCardPro #
#                    ject\EWARM\STM32Cube_SDCardProject                       #
#                    Configuration\Obj\stm32f1xx_ll_sdmmc.o"                  #
#                    "D:\Projects\MicroTechnics\STM32Cube\STM32Cube_SDCardPro #
#                    ject\EWARM\STM32Cube_SDCardProject                       #
#                    Configuration\Obj\syscall.o"                             #
#                    "D:\Projects\MicroTechnics\STM32Cube\STM32Cube_SDCardPro #
#                    ject\EWARM\STM32Cube_SDCardProject                       #
#                    Configuration\Obj\system_stm32f1xx.o" --redirect         #
#                    _Printf=_PrintfFull --redirect _Scanf=_ScanfFull -o      #
#                    "D:\Projects\MicroTechnics\STM32Cube\STM32Cube_SDCardPro #
#                    ject\EWARM\STM32Cube_SDCardProject                       #
#                    Configuration\Exe\STM32Cube_SDCardProject                #
#                    Configuration.out" --map "D:\Projects\MicroTechnics\STM3 #
#                    2Cube\STM32Cube_SDCardProject\EWARM\STM32Cube_SDCardProj #
#                    ect Configuration/List\STM32Cube_SDCardProject           #
#                    Configuration.map" --config "C:\Program Files (x86)\IAR  #
#                    Systems\Embedded Workbench 6.5\arm\config\linker\ST\stm3 #
#                    2f103xE.icf" --semihosting --entry __iar_program_start   #
#                    --vfe                                                    #
#                                                                             #
#                                                                             #
###############################################################################

*******************************************************************************
*** RUNTIME MODEL ATTRIBUTES
***

CppFlavor       = *
__Heap_Handler  = DLMalloc
__SystemLibrary = DLib


*******************************************************************************
*** PLACEMENT SUMMARY
***

"A1":  place at 0x08000000 { ro section .intvec };
"P1":  place in [from 0x08000000 to 0x0807ffff] { ro };
"P2":  place in [from 0x20000000 to 0x2000ffff] { rw, block CSTACK, block HEAP };

  Section            Kind        Address    Size  Object
  -------            ----        -------    ----  ------
"A1":                                      0x130
  .intvec            ro code  0x08000000   0x130  startup_stm32f103xe.o [1]
                            - 0x08000130   0x130

"P1":                                     0x6954
  .text              ro code  0x08000130  0x1f5c  ff.o [1]
  .text              ro code  0x0800208c    0xc8  diskio.o [1]
  .text              ro code  0x08002154    0x90  ccsbcs.o [1]
  .text              ro code  0x080021e4    0x18  syscall.o [1]
  .text              ro code  0x080021fc  0x14b4  dlmalloc.o [3]
  .text              ro code  0x080036b0     0x6  abort.o [3]
  .text              ro code  0x080036b6    0x2e  copy_init3.o [4]
  .text              ro code  0x080036e4    0x2c  xgetmemchunk.o [3]
  .text              ro code  0x08003710    0x14  exit.o [5]
  .text              ro code  0x08003724  0x1508  stm32f1xx_hal_sd.o [1]
  .text              ro code  0x08004c2c     0x6  ABImemclr4.o [4]
  .text              ro code  0x08004c32    0x22  zero_init3.o [4]
  .text              ro code  0x08004c54    0x90  stm32f1xx_hal_msp.o [1]
  .text              ro code  0x08004ce4    0x56  ABImemcpy_unaligned.o [4]
  .rodata            const    0x08004d3a     0x2  stm32f1xx_hal_rcc.o [1]
  .text              ro code  0x08004d3c    0xc0  stm32f1xx_ll_sdmmc.o [1]
  .text              ro code  0x08004dfc    0x7c  stm32f1xx_hal.o [1]
  .text              ro code  0x08004e78    0x32  ABImemset48.o [4]
  .text              ro code  0x08004eac   0x11e  stm32f1xx_hal_cortex.o [1]
  .text              ro code  0x08004fcc   0x320  stm32f1xx_hal_gpio.o [1]
  .text              ro code  0x080052ec   0x898  stm32f1xx_hal_rcc.o [1]
  .text              ro code  0x08005b84   0x390  stm32f1xx_hal_rcc_ex.o [1]
  .rodata            const    0x08005f14   0x1e0  ccsbcs.o [1]
  .rodata            const    0x080060f4   0x1e0  ccsbcs.o [1]
  .text              ro code  0x080062d4   0x15c  main.o [1]
  .text              ro code  0x08006430    0x54  ff_gen_drv.o [1]
  .text              ro code  0x08006484   0x114  sd_diskio.o [1]
  .text              ro code  0x08006598    0xd0  bsp_driver_sd.o [1]
  .rodata            const    0x08006668   0x100  ccsbcs.o [1]
  .rodata            const    0x08006768    0x80  ff.o [1]
  .text              ro code  0x080067e8    0x68  system_stm32f1xx.o [1]
  .text              ro code  0x08006850    0x28  data_init.o [4]
  .iar.init_table    const    0x08006878    0x24  - Linker created -
  .text              ro code  0x0800689c    0x1a  cmain.o [4]
  .text              ro code  0x080068b6     0x4  low_level_init.o [3]
  .text              ro code  0x080068ba     0x4  exit.o [3]
  .text              ro code  0x080068c0     0xa  cexit.o [4]
  .rodata            const    0x080068cc    0x10  ff.o [1]
  .rodata            const    0x080068dc    0x10  main.o [1]
  .rodata            const    0x080068ec    0x10  main.o [1]
  .rodata            const    0x080068fc    0x10  stm32f1xx_hal_rcc.o [1]
  .rodata            const    0x0800690c    0x10  stm32f1xx_hal_rcc.o [1]
  .text              ro code  0x0800691c    0x10  startup_stm32f103xe.o [1]
  .rodata            const    0x0800692c     0xc  ff.o [1]
  .text              ro code  0x08006938     0xc  stm32f1xx_it.o [1]
  .text              ro code  0x08006944     0xc  cstartup_M.o [4]
  .rodata            const    0x08006950     0x8  ff.o [1]
  .text              ro code  0x08006958     0x4  startup_stm32f103xe.o [1]
  .text              ro code  0x0800695c     0x4  startup_stm32f103xe.o [1]
  .text              ro code  0x08006960     0x4  startup_stm32f103xe.o [1]
  .text              ro code  0x08006964     0x4  startup_stm32f103xe.o [1]
  .text              ro code  0x08006968     0x4  startup_stm32f103xe.o [1]
  .text              ro code  0x0800696c     0x4  startup_stm32f103xe.o [1]
  .text              ro code  0x08006970     0x4  startup_stm32f103xe.o [1]
  .text              ro code  0x08006974     0x4  startup_stm32f103xe.o [1]
  .text              ro code  0x08006978     0x4  startup_stm32f103xe.o [1]
  .text              ro code  0x0800697c     0x4  startup_stm32f103xe.o [1]
  .text              ro code  0x08006980     0x4  startup_stm32f103xe.o [1]
  .text              ro code  0x08006984     0x4  startup_stm32f103xe.o [1]
  .text              ro code  0x08006988     0x4  startup_stm32f103xe.o [1]
  .text              ro code  0x0800698c     0x4  startup_stm32f103xe.o [1]
  .text              ro code  0x08006990     0x4  startup_stm32f103xe.o [1]
  .text              ro code  0x08006994     0x4  startup_stm32f103xe.o [1]
  .text              ro code  0x08006998     0x4  startup_stm32f103xe.o [1]
  .text              ro code  0x0800699c     0x4  startup_stm32f103xe.o [1]
  .text              ro code  0x080069a0     0x4  startup_stm32f103xe.o [1]
  .text              ro code  0x080069a4     0x4  startup_stm32f103xe.o [1]
  .text              ro code  0x080069a8     0x4  startup_stm32f103xe.o [1]
  .text              ro code  0x080069ac     0x4  startup_stm32f103xe.o [1]
  .text              ro code  0x080069b0     0x4  startup_stm32f103xe.o [1]
  .text              ro code  0x080069b4     0x4  startup_stm32f103xe.o [1]
  .text              ro code  0x080069b8     0x4  startup_stm32f103xe.o [1]
  .text              ro code  0x080069bc     0x4  startup_stm32f103xe.o [1]
  .text              ro code  0x080069c0     0x4  startup_stm32f103xe.o [1]
  .text              ro code  0x080069c4     0x4  startup_stm32f103xe.o [1]
  .text              ro code  0x080069c8     0x4  startup_stm32f103xe.o [1]
  .text              ro code  0x080069cc     0x4  startup_stm32f103xe.o [1]
  .text              ro code  0x080069d0     0x4  startup_stm32f103xe.o [1]
  .text              ro code  0x080069d4     0x4  startup_stm32f103xe.o [1]
  .text              ro code  0x080069d8     0x4  startup_stm32f103xe.o [1]
  .text              ro code  0x080069dc     0x4  startup_stm32f103xe.o [1]
  .text              ro code  0x080069e0     0x4  startup_stm32f103xe.o [1]
  .text              ro code  0x080069e4     0x4  startup_stm32f103xe.o [1]
  .text              ro code  0x080069e8     0x4  startup_stm32f103xe.o [1]
  .text              ro code  0x080069ec     0x4  startup_stm32f103xe.o [1]
  .text              ro code  0x080069f0     0x4  startup_stm32f103xe.o [1]
  .text              ro code  0x080069f4     0x4  startup_stm32f103xe.o [1]
  .text              ro code  0x080069f8     0x4  startup_stm32f103xe.o [1]
  .text              ro code  0x080069fc     0x4  startup_stm32f103xe.o [1]
  .text              ro code  0x08006a00     0x4  startup_stm32f103xe.o [1]
  .text              ro code  0x08006a04     0x4  startup_stm32f103xe.o [1]
  .text              ro code  0x08006a08     0x4  startup_stm32f103xe.o [1]
  .text              ro code  0x08006a0c     0x4  startup_stm32f103xe.o [1]
  .text              ro code  0x08006a10     0x4  startup_stm32f103xe.o [1]
  .text              ro code  0x08006a14     0x4  startup_stm32f103xe.o [1]
  .text              ro code  0x08006a18     0x4  startup_stm32f103xe.o [1]
  .text              ro code  0x08006a1c     0x4  startup_stm32f103xe.o [1]
  .text              ro code  0x08006a20     0x4  startup_stm32f103xe.o [1]
  .text              ro code  0x08006a24     0x4  startup_stm32f103xe.o [1]
  .text              ro code  0x08006a28     0x4  startup_stm32f103xe.o [1]
  .text              ro code  0x08006a2c     0x4  startup_stm32f103xe.o [1]
  .text              ro code  0x08006a30     0x4  startup_stm32f103xe.o [1]
  .text              ro code  0x08006a34     0x4  startup_stm32f103xe.o [1]
  .text              ro code  0x08006a38     0x4  startup_stm32f103xe.o [1]
  .text              ro code  0x08006a3c     0x4  startup_stm32f103xe.o [1]
  .text              ro code  0x08006a40     0x4  startup_stm32f103xe.o [1]
  .text              ro code  0x08006a44     0x4  startup_stm32f103xe.o [1]
  .text              ro code  0x08006a48     0x4  startup_stm32f103xe.o [1]
  .text              ro code  0x08006a4c     0x4  startup_stm32f103xe.o [1]
  .text              ro code  0x08006a50     0x4  startup_stm32f103xe.o [1]
  .text              ro code  0x08006a54     0x4  startup_stm32f103xe.o [1]
  .text              ro code  0x08006a58     0x4  startup_stm32f103xe.o [1]
  .text              ro code  0x08006a5c     0x4  startup_stm32f103xe.o [1]
  .text              ro code  0x08006a60     0x4  startup_stm32f103xe.o [1]
  .text              ro code  0x08006a64     0x4  startup_stm32f103xe.o [1]
  .rodata            const    0x08006a68     0x0  zero_init3.o [4]
  .rodata            const    0x08006a68     0x0  copy_init3.o [4]
  Initializer bytes  ro data  0x08006a68    0x1c  <for P2 s0>
                            - 0x08006a84  0x6954

"P2", part 1 of 3:                          0x1c
  P2 s0                       0x20000000    0x1c  <Init block>
    .data            inited   0x20000000    0x14  sd_diskio.o [1]
    .data            inited   0x20000014     0x4  system_stm32f1xx.o [1]
    .data            inited   0x20000018     0x1  sd_diskio.o [1]
                            - 0x2000001c    0x1c

"P2", part 2 of 3:                         0x2e4
  .bss               zero     0x2000001c   0x1d8  dlmalloc.o [3]
  .bss               zero     0x200001f4    0x60  main.o [1]
  .bss               zero     0x20000258    0x58  main.o [1]
  .bss               zero     0x200002b0    0x18  ff.o [1]
  .bss               zero     0x200002c8    0x18  dlmalloc.o [3]
  .bss               zero     0x200002e0     0xc  ff_gen_drv.o [1]
  .bss               zero     0x200002ec     0x4  ff.o [1]
  .bss               zero     0x200002f0     0x4  main.o [1]
  .bss               zero     0x200002f4     0x4  stm32f1xx_hal.o [1]
  .bss               zero     0x200002f8     0x4  xgetmemchunk.o [3]
  .bss               zero     0x200002fc     0x2  ff.o [1]
  .bss               zero     0x200002fe     0x1  main.o [1]
  .bss               zero     0x200002ff     0x1  main.o [1]
                            - 0x20000300   0x2e4

"P2", part 3 of 3:                        0x2000
  CSTACK                      0x20000300  0x1000  <Block>
    CSTACK           uninit   0x20000300  0x1000  <Block tail>
  HEAP                        0x20001300  0x1000  <Block>
    HEAP             uninit   0x20001300  0x1000  <Block tail>
                            - 0x20002300  0x2000


*******************************************************************************
*** INIT TABLE
***

          Address     Size
          -------     ----
Zero (__iar_zero_init3)
    1 destination range, total size 0x2e4:
          0x2000001c  0x2e4

Copy (__iar_copy_init3)
    1 source range, total size 0x1c (112% of destination):
          0x08006a68   0x1c
    1 destination range, total size 0x19:
          0x20000000   0x19



*******************************************************************************
*** MODULE SUMMARY
***

    Module                  ro code  ro data  rw data
    ------                  -------  -------  -------
D:\Projects\MicroTechnics\STM32Cube\STM32Cube_SDCardProject\EWARM\STM32Cube_SDCardProject Configuration\Obj: [1]
    bsp_driver_sd.o             208
    ccsbcs.o                    144    1 216
    diskio.o                    200
    ff.o                      8 028      164       30
    ff_gen_drv.o                 84                12
    main.o                      348       32      190
    sd_diskio.o                 276       21       21
    startup_stm32f103xe.o       592
    stm32f1xx_hal.o             124                 4
    stm32f1xx_hal_cortex.o      286
    stm32f1xx_hal_gpio.o        800
    stm32f1xx_hal_msp.o         144
    stm32f1xx_hal_rcc.o       2 200       34
    stm32f1xx_hal_rcc_ex.o      912
    stm32f1xx_hal_sd.o        5 384
    stm32f1xx_it.o               12
    stm32f1xx_ll_sdmmc.o        192
    syscall.o                    24
    system_stm32f1xx.o          104        4        4
    -------------------------------------------------
    Total:                   20 062    1 471      261

command line: [2]
    -------------------------------------------------
    Total:

dl7M_tlf.a: [3]
    abort.o                       6
    dlmalloc.o                5 300               496
    exit.o                        4
    low_level_init.o              4
    xgetmemchunk.o               44                 4
    -------------------------------------------------
    Total:                    5 358               500

rt7M_tl.a: [4]
    ABImemclr4.o                  6
    ABImemcpy_unaligned.o        86
    ABImemset48.o                50
    cexit.o                      10
    cmain.o                      26
    copy_init3.o                 46
    cstartup_M.o                 12
    data_init.o                  40
    zero_init3.o                 34
    -------------------------------------------------
    Total:                      310

shb_l.a: [5]
    exit.o                       20
    -------------------------------------------------
    Total:                       20

    Gaps                          6        2        4
    Linker created                        39    8 192
-----------------------------------------------------
    Grand Total:             25 756    1 512    8 957


*******************************************************************************
*** ENTRY LIST
***

Entry                      Address   Size  Type      Object
-----                      -------   ----  ----      ------
?main                   0x0800689d         Code  Gb  cmain.o [4]
BSP_SD_GetCardInfo      0x08006641    0xe  Code  Gb  bsp_driver_sd.o [1]
BSP_SD_GetStatus        0x08006637    0xa  Code  Gb  bsp_driver_sd.o [1]
BSP_SD_Init             0x08006599   0x3e  Code  Gb  bsp_driver_sd.o [1]
BSP_SD_IsDetected       0x08006659   0x10  Code  Gb  bsp_driver_sd.o [1]
BSP_SD_ReadBlocks       0x080065d7   0x30  Code  Gb  bsp_driver_sd.o [1]
BSP_SD_WriteBlocks      0x08006607   0x30  Code  Gb  bsp_driver_sd.o [1]
CSTACK$$Base            0x20000300          --   Gb  - Linker created -
CSTACK$$Limit           0x20001300          --   Gb  - Linker created -
ExCvt                   0x08006768   0x80  Data  Lc  ff.o [1]
FATFS_LinkDriver        0x08006431   0x4e  Code  Gb  ff_gen_drv.o [1]
FatFs                   0x200002ec    0x4  Data  Lc  ff.o [1]
Files                   0x200002b0   0x18  Data  Lc  ff.o [1]
Fsid                    0x200002fc    0x2  Data  Lc  ff.o [1]
HAL_Delay               0x08004e55   0x1a  Code  Wk  stm32f1xx_hal.o [1]
HAL_GPIO_Init           0x08004fcd  0x2d6  Code  Gb  stm32f1xx_hal_gpio.o [1]
HAL_GetTick             0x08004e4f    0x6  Code  Wk  stm32f1xx_hal.o [1]
HAL_IncTick             0x08004e43    0xc  Code  Wk  stm32f1xx_hal.o [1]
HAL_Init                0x08004dfd   0x22  Code  Gb  stm32f1xx_hal.o [1]
HAL_InitTick            0x08004e1f   0x24  Code  Wk  stm32f1xx_hal.o [1]
HAL_MspInit             0x08004c55   0x26  Code  Gb  stm32f1xx_hal_msp.o [1]
HAL_NVIC_SetPriority    0x08004f71   0x26  Code  Gb  stm32f1xx_hal_cortex.o [1]
HAL_NVIC_SetPriorityGrouping
                        0x08004f65    0xc  Code  Gb  stm32f1xx_hal_cortex.o [1]
HAL_RCC_ClockConfig     0x08005b85  0x380  Code  Gb  stm32f1xx_hal_rcc_ex.o [1]
HAL_RCC_GetHCLKFreq     0x08005b1d   0x28  Code  Gb  stm32f1xx_hal_rcc.o [1]
HAL_RCC_GetSysClockFreq
                        0x08005a93   0x8a  Code  Wk  stm32f1xx_hal_rcc.o [1]
HAL_RCC_OscConfig       0x080052ed  0x7a6  Code  Wk  stm32f1xx_hal_rcc.o [1]
HAL_SD_GetStatus        0x080040f3   0x26  Code  Gb  stm32f1xx_hal_sd.o [1]
HAL_SD_Get_CardInfo     0x08003cc7  0x350  Code  Gb  stm32f1xx_hal_sd.o [1]
HAL_SD_Init             0x08003725   0xba  Code  Gb  stm32f1xx_hal_sd.o [1]
HAL_SD_MspInit          0x08004c7b   0x54  Code  Gb  stm32f1xx_hal_msp.o [1]
HAL_SD_ReadBlocks       0x080037df  0x222  Code  Gb  stm32f1xx_hal_sd.o [1]
HAL_SD_StopTransfer     0x080040b3   0x40  Code  Gb  stm32f1xx_hal_sd.o [1]
HAL_SD_WideBusOperation_Config
                        0x08004017   0x9c  Code  Gb  stm32f1xx_hal_sd.o [1]
HAL_SD_WriteBlocks      0x08003a01  0x2c6  Code  Gb  stm32f1xx_hal_sd.o [1]
HAL_SYSTICK_Callback    0x08004fc9    0x2  Code  Wk  stm32f1xx_hal_cortex.o [1]
HAL_SYSTICK_Config      0x08004f97    0xc  Code  Gb  stm32f1xx_hal_cortex.o [1]
HAL_SYSTICK_IRQHandler  0x08004fc1    0x8  Code  Gb  stm32f1xx_hal_cortex.o [1]
HEAP$$Base              0x20001300          --   Gb  - Linker created -
HEAP$$Limit             0x20002300          --   Gb  - Linker created -
LfnOfs                  0x080068cc   0x10  Data  Lc  ff.o [1]
MX_GPIO_Init            0x080063d7   0x36  Code  Lc  main.o [1]
MX_SDIO_SD_Init         0x080063ab   0x2c  Code  Lc  main.o [1]
NVIC_EncodePriority     0x08004ef7   0x3e  Code  Lc  stm32f1xx_hal_cortex.o [1]
NVIC_GetPriorityGrouping
                        0x08004ecb    0xa  Code  Lc  stm32f1xx_hal_cortex.o [1]
NVIC_SetPriority        0x08004ed5   0x22  Code  Lc  stm32f1xx_hal_cortex.o [1]
NVIC_SetPriorityGrouping
                        0x08004ead   0x1e  Code  Lc  stm32f1xx_hal_cortex.o [1]
Region$$Table$$Base     0x08006878          --   Gb  - Linker created -
Region$$Table$$Limit    0x0800689c          --   Gb  - Linker created -
SDCardInfo              0x20000258   0x58  Data  Gb  main.o [1]
SDIO_DataConfig         0x08004dcd   0x26  Code  Gb  stm32f1xx_ll_sdmmc.o [1]
SDIO_GetCommandResponse
                        0x08004db1    0x6  Code  Gb  stm32f1xx_ll_sdmmc.o [1]
SDIO_GetPowerState      0x08004d83    0x8  Code  Gb  stm32f1xx_ll_sdmmc.o [1]
SDIO_GetResponse        0x08004db7   0x16  Code  Gb  stm32f1xx_ll_sdmmc.o [1]
SDIO_Init               0x08004d3d   0x2a  Code  Gb  stm32f1xx_ll_sdmmc.o [1]
SDIO_PowerState_ON      0x08004d79    0xa  Code  Gb  stm32f1xx_ll_sdmmc.o [1]
SDIO_ReadFIFO           0x08004d67    0x6  Code  Gb  stm32f1xx_ll_sdmmc.o [1]
SDIO_SendCommand        0x08004d8b   0x26  Code  Gb  stm32f1xx_ll_sdmmc.o [1]
SDIO_WriteFIFO          0x08004d6d    0xc  Code  Gb  stm32f1xx_ll_sdmmc.o [1]
SD_CmdError             0x0800449f   0x4c  Code  Lc  stm32f1xx_hal_sd.o [1]
SD_CmdResp1Error        0x08004565  0x118  Code  Lc  stm32f1xx_hal_sd.o [1]
SD_CmdResp2Error        0x080046ad   0x46  Code  Lc  stm32f1xx_hal_sd.o [1]
SD_CmdResp3Error        0x0800467d   0x30  Code  Lc  stm32f1xx_hal_sd.o [1]
SD_CmdResp6Error        0x080046f3   0xaa  Code  Lc  stm32f1xx_hal_sd.o [1]
SD_CmdResp7Error        0x080044eb   0x7a  Code  Lc  stm32f1xx_hal_sd.o [1]
SD_Driver               0x20000000   0x14  Data  Gb  sd_diskio.o [1]
SD_FindSCR              0x08004911  0x1a0  Code  Lc  stm32f1xx_hal_sd.o [1]
SD_GetState             0x08004119   0x24  Code  Lc  stm32f1xx_hal_sd.o [1]
SD_Initialize_Cards     0x0800413d  0x130  Code  Lc  stm32f1xx_hal_sd.o [1]
SD_IsCardProgramming    0x08004ab1  0x174  Code  Lc  stm32f1xx_hal_sd.o [1]
SD_Path                 0x200002f0    0x4  Data  Gb  main.o [1]
SD_PowerON              0x080042af  0x188  Code  Lc  stm32f1xx_hal_sd.o [1]
SD_Select_Deselect      0x0800426d   0x42  Code  Lc  stm32f1xx_hal_sd.o [1]
SD_SendStatus           0x08004437   0x68  Code  Lc  stm32f1xx_hal_sd.o [1]
SD_WideBus_Disable      0x08004857   0xba  Code  Lc  stm32f1xx_hal_sd.o [1]
SD_WideBus_Enable       0x0800479d   0xba  Code  Lc  stm32f1xx_hal_sd.o [1]
SD_initialize           0x08006485   0x22  Code  Gb  sd_diskio.o [1]
SD_ioctl                0x0800652d   0x68  Code  Gb  sd_diskio.o [1]
SD_read                 0x080064c9   0x32  Code  Gb  sd_diskio.o [1]
SD_status               0x080064a7   0x22  Code  Gb  sd_diskio.o [1]
SD_write                0x080064fb   0x32  Code  Gb  sd_diskio.o [1]
Stat                    0x20000018    0x1  Data  Lc  sd_diskio.o [1]
SysTick_Config          0x08004f35   0x30  Code  Lc  stm32f1xx_hal_cortex.o [1]
SysTick_Handler         0x08006939    0xc  Code  Gb  stm32f1xx_it.o [1]
SystemClock_Config      0x08006357   0x54  Code  Gb  main.o [1]
SystemCoreClock         0x20000014    0x4  Data  Gb  system_stm32f1xx.o [1]
SystemInit              0x080067e9   0x4e  Code  Gb  system_stm32f1xx.o [1]
Tbl                     0x08006668  0x100  Data  Lc  ccsbcs.o [1]
__aeabi_memclr4         0x08004c2d         Code  Gb  ABImemclr4.o [4]
__cmain                 0x0800689d         Code  Gb  cmain.o [4]
__data_GetMemChunk      0x080036e5   0x2c  Code  Gb  xgetmemchunk.o [3]
__exit                  0x08003711   0x14  Code  Gb  exit.o [5]
__iar_Memset4_word      0x08004e79         Code  Gb  ABImemset48.o [4]
__iar_Memset8_word      0x08004e79         Code  Gb  ABImemset48.o [4]
__iar_copy_init3        0x080036b7   0x2e  Code  Gb  copy_init3.o [4]
__iar_data_init3        0x08006851   0x28  Code  Gb  data_init.o [4]
__iar_dlfree            0x08003195  0x512  Code  Gb  dlmalloc.o [3]
__iar_dlmalloc          0x08002ee1  0x2a8  Code  Gb  dlmalloc.o [3]
__iar_gm_               0x2000001c  0x1d8  Data  Gb  dlmalloc.o [3]
__iar_program_start     0x08006945         Code  Gb  cstartup_M.o [4]
__iar_unaligned___aeabi_memcpy4
                        0x08004ce5         Code  Gb  ABImemcpy_unaligned.o [4]
__iar_unaligned___aeabi_memcpy8
                        0x08004ce5         Code  Gb  ABImemcpy_unaligned.o [4]
__iar_zero_init3        0x08004c33   0x22  Code  Gb  zero_init3.o [4]
__low_level_init        0x080068b7    0x4  Code  Gb  low_level_init.o [3]
__vector_table          0x08000000         Data  Gb  startup_stm32f103xe.o [1]
_call_main              0x080068a9         Code  Gb  cmain.o [4]
_exit                   0x080068c1         Code  Gb  cexit.o [4]
_main                   0x080068b3         Code  Gb  cmain.o [4]
aAPBAHBPrescTable       0x0800690c   0x10  Data  Gb  stm32f1xx_hal_rcc.o [1]
abort                   0x080036b1    0x6  Code  Gb  abort.o [3]
check_fs                0x08001509   0x82  Code  Lc  ff.o [1]
chk_chr                 0x08000187   0x14  Code  Lc  ff.o [1]
chk_lock                0x0800019b   0x9a  Code  Lc  ff.o [1]
clear_lock              0x080003ad   0x2c  Code  Lc  ff.o [1]
clmt_clust              0x08000971   0x3e  Code  Lc  ff.o [1]
clust2sect              0x08000561   0x20  Code  Gb  ff.o [1]
cmp_lfn                 0x08000cb3   0x9e  Code  Lc  ff.o [1]
create_chain            0x08000873   0xfe  Code  Lc  ff.o [1]
create_name             0x08001165  0x2b8  Code  Lc  ff.o [1]
dec_lock                0x08000351   0x5c  Code  Lc  ff.o [1]
dir_alloc               0x08000c03   0x6e  Code  Lc  ff.o [1]
dir_find                0x08000ec1  0x12e  Code  Lc  ff.o [1]
dir_next                0x08000a8b  0x178  Code  Lc  ff.o [1]
dir_register            0x08000fef  0x176  Code  Lc  ff.o [1]
dir_sdi                 0x080009af   0xdc  Code  Lc  ff.o [1]
disk                    0x200002e0    0xc  Data  Gb  ff_gen_drv.o [1]
disk_initialize         0x0800208d   0x2e  Code  Gb  diskio.o [1]
disk_ioctl              0x08002129   0x24  Code  Gb  diskio.o [1]
disk_read               0x080020d5   0x2a  Code  Gb  diskio.o [1]
disk_status             0x080020bb   0x1a  Code  Gb  diskio.o [1]
disk_write              0x080020ff   0x2a  Code  Gb  diskio.o [1]
enq_lock                0x08000235   0x28  Code  Lc  ff.o [1]
exit                    0x080068bb    0x4  Code  Gb  exit.o [3]
f_close                 0x08002051   0x3c  Code  Gb  ff.o [1]
f_mount                 0x08001a17   0x6a  Code  Gb  ff.o [1]
f_open                  0x08001aa1  0x224  Code  Gb  ff.o [1]
f_sync                  0x08001f75   0xdc  Code  Gb  ff.o [1]
f_write                 0x08001cc5  0x2b0  Code  Gb  ff.o [1]
ff_convert              0x08002155   0x4e  Code  Gb  ccsbcs.o [1]
ff_memalloc             0x080021e5    0xc  Code  Gb  syscall.o [1]
ff_memfree              0x080021f1    0xc  Code  Gb  syscall.o [1]
ff_wtoupper             0x080021a3   0x34  Code  Gb  ccsbcs.o [1]
find_volume             0x08001591  0x43c  Code  Lc  ff.o [1]
fit_lfn                 0x08000d51   0x84  Code  Lc  ff.o [1]
follow_path             0x0800141d   0x9c  Code  Lc  ff.o [1]
gen_numname             0x08000dd9   0xca  Code  Lc  ff.o [1]
get_fat                 0x08000581  0x102  Code  Gb  ff.o [1]
get_fattime             0x08002151    0x4  Code  Gb  diskio.o [1]
get_ldnumber            0x080014b9   0x50  Code  Lc  ff.o [1]
hsd                     0x200001f4   0x60  Data  Gb  main.o [1]
inc_lock                0x0800025d   0xf4  Code  Lc  ff.o [1]
init_mparams            0x08002217   0x34  Code  Lc  dlmalloc.o [3]
init_top                0x0800224b   0x34  Code  Lc  dlmalloc.o [3]
ld_clust                0x08000c71   0x2a  Code  Lc  ff.o [1]
main                    0x080062d5   0x82  Code  Gb  main.o [1]
mem_cmp                 0x08000163   0x24  Code  Lc  ff.o [1]
mem_cpy                 0x08000131   0x1c  Code  Lc  ff.o [1]
mem_set                 0x0800014d   0x16  Code  Lc  ff.o [1]
move_window             0x0800043b   0x3a  Code  Lc  ff.o [1]
mparams                 0x200002c8   0x18  Data  Lc  dlmalloc.o [3]
prepend_alloc           0x0800227f  0x33c  Code  Lc  dlmalloc.o [3]
put_fat                 0x08000683  0x16c  Code  Gb  ff.o [1]
remove_chain            0x080007ef   0x84  Code  Lc  ff.o [1]
res                     0x200002ff    0x1  Data  Gb  main.o [1]
retSD                   0x200002fe    0x1  Data  Gb  main.o [1]
segment_holding         0x080021fd   0x1a  Code  Lc  dlmalloc.o [3]
st_clust                0x08000c9b   0x18  Code  Lc  ff.o [1]
sum_sfn                 0x08000ea3   0x1e  Code  Lc  ff.o [1]
sync_fs                 0x08000475   0xec  Code  Lc  ff.o [1]
sync_window             0x080003d9   0x62  Code  Lc  ff.o [1]
sys_alloc               0x080025bb  0x37e  Code  Lc  dlmalloc.o [3]
tmalloc_large           0x08002945  0x38a  Code  Lc  dlmalloc.o [3]
tmalloc_small           0x08002ccf  0x204  Code  Lc  dlmalloc.o [3]
uwTick                  0x200002f4    0x4  Data  Lc  stm32f1xx_hal.o [1]
validate                0x080019cd   0x4a  Code  Lc  ff.o [1]


[1] = D:\Projects\MicroTechnics\STM32Cube\STM32Cube_SDCardProject\EWARM\STM32Cube_SDCardProject Configuration\Obj
[2] = command line
[3] = dl7M_tlf.a
[4] = rt7M_tl.a
[5] = shb_l.a

  25 756 bytes of readonly  code memory
   1 512 bytes of readonly  data memory
   8 957 bytes of readwrite data memory

Errors: none
Warnings: none
